:100000000C94C7010C94EF010C94EF010C94EF01D8
:100010000C94EF010C94EF010C94EF010C94EF01A0
:100020000C94EF010C94EF010C94EF010C94EF0190
:100030000C94EF010C94EF010C94EF010C94EF0180
:100040000C94D11D0C94EF010C94A01F0C94EF01A3
:100050000C94EF010C94EF010C94EF010C94EF0160
:100060000C94521A0C94EF0100000000003F484825
:10007000483F7F494949363E414141227F41412223
:100080001C7F494949417F484848403E4149492EE3
:100090007F0808087F00417F4100060101017E7F43
:1000A000081422417F010101017F2010207F7F1071
:1000B00008047F3E4141413E7F484848303E41452B
:1000C000423D7F484C4A31314949494640407F4092
:1000D000407E0101017E7C0201027C7F0204027FDE
:1000E000631408146360100F1060434549516101A7
:1000F00000000000000070000000001400007F22DB
:100100001408003E4549513E00217F01002143452E
:10011000493122414949360C14247F04725151510E
:100120004E3E4949492640404F506036494949367C
:10013000324949493E000000000000000000000074
:1001400000000000000000000000000000000000AF
:10015000000000000000000000000000000000009F
:10016000000000000000003F7FE0C1C3C7CEFC7F5D
:100170003FF0F8FCCC8C0C0C3CF8F000003070FF29
:10018000FF0000000000000C0CFCFC0C0C00003018
:1001900070E0C0C0C1C3E77E3C0C1C3C7CECCC8C46
:1001A0000C0C0C3070E0C0C0C3C3E37F3C30381C83
:1001B0000C0C0C0C1CF8F003070E1C3870FFFF0031
:1001C00000C0C0C0C0C0C0FCFCC0C0FCFCCCCCCCDB
:1001D000CCCCCEC7C330381C0C0C0C0C1CF8F03F38
:1001E0007FE3C3C3C3C3E36120F0F81C0C0C0C0C09
:1001F0009CF8F0C0C0C0C1C3C7CEDCF8F00000005E
:10020000FCFC00000000003C7FE7C3C3C3C3E77FE2
:100210003CF0F89C0C0C0C0C9CF8F03C7EE7C3C343
:10022000C3C3C37F3F10181C0C0C0C0C1CF8F0004F
:1002300000000000001F0014001F001F0015000A2E
:10024000001F00110011001F0011000E001F0015FB
:100250000011001F00140010001F00110017001FE4
:100260000004001F0011001F001100030001001F07
:10027000001F0004001B001F00010001001F0008F8
:10028000001F001F0010000F001F0011001F001FA3
:100290000014001C001C0014001F001F0016001D8D
:1002A000001D001500170010001F0010001F0001A6
:1002B000001F001E0001001E001F0002001F001B87
:1002C0000004001B001C0007001C0013001500198F
:1002D000000100000000001800000000001D0000E8
:1002E000000000100015001C001F0011001F00007E
:1002F0000000001F00170015001D00110015001F51
:10030000001C0004001F001D00150017001F001531
:10031000001700100010001F001F0015001F001D17
:100320000015001F00000000000000000000002475
:100330000027002A0000000000250028002B0000F4
:10034000000000230026002900040404040404041F
:100350000402020202020203030303030301020474
:100360000810204080010204081020010204081037
:100370002000000007000201000003040600000046
:10038000000000000000F60257196C1D9C2011248B
:100390001FBECFEFD8E0DEBFCDBF13E0A0E0B1E0DD
:1003A000E4EFF6E402C005900D92A63EB107D9F73E
:1003B00016E0A6EEB3E001C01D92AC31B107E1F743
:1003C00013E0CEE8D3E004C02297FE010E943D2353
:1003D000C638D107C9F70E94D6200C9478230C9414
:1003E0000000A0E0B0E0E7EFF1E00C944923EC015D
:1003F000A880B980CA80DB80A114B104C104D104F3
:1004000041F484E2A82E89EDB82E8BE5C82E87E052
:10041000D82EC601B5012DE133EF41E050E00E9436
:100420000C2327EA31E440E050E00E94AC227B013B
:100430008C01C601B5012DE133EF41E050E00E948F
:100440000C23CA01B9012CEE34EF4FEF5FEF0E948D
:10045000AC226E0D7F1D801F911F97FF04C061505D
:10046000704080409048688379838A839B839B0196
:100470003F77C901CDB7DEB7EAE00C9465230E944F
:10048000F101089580E493E00E94F1010895A0E055
:10049000B0E08093400390934103A0934203B09354
:1004A00043030895A0E0B0E0E8E5F2E00C944923AE
:1004B000EC01A880B980CA80DB80A114B104C1041A
:1004C000D10441F484E2A82E89EDB82E8BE5C82E24
:1004D00087E0D82EC601B5012DE133EF41E050E0B1
:1004E0000E940C2327EA31E440E050E00E94AC2255
:1004F0007B018C01C601B5012DE133EF41E050E0F5
:100500000E940C23CA01B9012CEE34EF4FEF5FEFCC
:100510000E94AC226E0D7F1D801F911F97FF04C0AB
:100520006150704080409048688379838A839B83C0
:100530009B01AC015F77B901CA01CDB7DEB7EAE034
:100540000C9465230E945202089584E493E00E9473
:1005500052020895609344037093450380934603C9
:10056000909347030895FB01DC010D900020E9F70B
:10057000119701900D920020E1F70895FB01DC0135
:1005800001900D920020E1F70895FB019F01E8948E
:100590004230C4F04532B4F44A3029F497FB1EF4DB
:1005A000909581959F4F642F77270E942723805D28
:1005B0008A330CF0895D8193CB010097A1F716F483
:1005C0005DE251931082C9010C94E602DC01FC014A
:1005D000672F71917723E1F7329704C07C916D9377
:1005E00070836291AE17BF07C8F3089586EE93E05B
:1005F00062E041E00E94B41D89EE93E063E041E0D7
:100600000E94B41D80914803909149039093010486
:100610008093000408951F93CF93DF93162FC82F64
:10062000D0E016C08BE060E00E94F51E812F90E0C4
:100630008C239D23892B19F08AE061E002C08AE0B7
:1006400060E00E94F51E8BE061E00E94F51E1695A9
:10065000112341F7DF91CF911F91089561E00E942E
:10066000F51E089560E00E94F51E08950F931F93F4
:10067000162FEDE9F3E0E80FF11D0081802F0E94B5
:10068000320384E064E00E940B03812F60E80E9443
:100690000B0380E061E00E940B03802F0E942E0379
:1006A0001F910F910895EF92FF920F931F93CF9395
:1006B000DF93CDE9D3E0EE24FF240881802F0E9450
:1006C000320385E064E00E940B0380E060E40E9456
:1006D0000B0310E080E060E80E940B031F5F103303
:1006E000C9F7802F0E942E03F701EE5FFB4F80E0D9
:1006F00011928F5F8036E1F7219680E690E0E80E58
:10070000F91E93E0CF39D907C1F6DF91CF911F9140
:100710000F91FF90EF9008950F931F9300914C035A
:1007200011C0102F105680E0612F0E94360381E027
:10073000612F0E9436036EE170E080E090E00E943D
:10074000191E015007FFEDCF0E94530360914C0327
:10075000605680E00E94360360914C03605681E051
:100760000E9436031F910F910895FF920F931F93DC
:10077000062FF42EEDE9F3E0E80FF11D1081812F33
:100780000E94320385E064E00E940B03802F60E446
:100790000E940B038F2D68E00E940B03812F0E94A3
:1007A0002E031F910F91FF900895782FE42F282F8B
:1007B0002851283110F0A0E002C0722FA1E0862F4E
:1007C000992787FD9095AC014370507028E030E088
:1007D00002C0359527954A95E2F7672F660F660F99
:1007E0009595879595958795680F862F992787FD0D
:1007F0009095EE2359F0E0E6AE9FF0011124E80F4A
:10080000F91FEE5FFB4F8081822B0BC0E0E6AE9FAD
:10081000F0011124E80FF91FEE5FFB4F2095808156
:1008200082238083462F552747FD50952A2F30E09D
:1008300080E690E0289FF001299FF00D389FF00D91
:100840001124E40FF51FEE5FFB4F8A2F40810E94B9
:10085000B50308959F92AF92BF92CF92DF92EF922D
:10086000FF920F931F93982EA62EB42EC22ED02E39
:10087000EE243AC0612F6A0D8F2D41E00E94D5030E
:100880001F5FC116B8F70F5FB01620F010E0F02E12
:10089000F90CF0CFDD2029F060E971E080E090E014
:1008A00004C066E470E080E090E00E94191E00E061
:1008B0000CC0612F6A0D8F2D40E00E94D5031F5F91
:1008C000C116B8F70F5FB01620F010E0F02EF90C4B
:1008D000F0CFDD2031F060E971E080E090E00E942F
:1008E000191EE394DE1410F000E0D0CF1F910F9199
:1008F000FF90EF90DF90CF90BF90AF909F900895C2
:10090000BF92CF92DF92EF92FF920F931F93B82E78
:10091000C62ED42EE22E00E00CC0612F6C0D8F2D60
:1009200041E00E94D5031F5FE116B8F70F5FD016B4
:1009300020F010E0F02EFB0CF0CF1F910F91FF90F4
:10094000EF90DF90CF90BF9008957F928F929F920B
:10095000AF92BF92CF92DF92EF92FF920F931F93CD
:10096000CF93DF93E82E762E842F81548A3118F0AE
:1009700080528A3110F44F7119C0842F80538A300D
:1009800010F4415113C0403211F440E00FC04E3218
:1009900011F44BE10BC0473211F44CE107C0413276
:1009A00011F44DE103C04F3309F44EE100E010E0D3
:1009B00083E0480250011124B0E18B2E912CF80104
:1009C000EA0DFB1DEE0FFF1FE15DFD4FE491F72CDB
:1009D000C0E0D0E0CE2EDD24C4010C2E02C09595DF
:1009E00087950A94E2F78C219D21892B21F08E2D89
:1009F0006F2D41E003C08E2D6F2D40E00E94D50386
:100A00002196F394C530D10539F70F5F1F4FE3945A
:100A100003301105A1F6DF91CF911F910F91FF9047
:100A2000EF90DF90CF90BF90AF909F908F907F908E
:100A300008956F927F928F929F92AF92BF92CF92C2
:100A4000DF92EF92FF920F931F93CF93DF93082FC4
:100A5000762E842F81548A3108F46FC080528A31F7
:100A600008F46BC08F5C8A3010F4482F4F71EE246D
:100A7000FF24242F332727FD309584E190E0289F21
:100A80005001299FB00C389FB00C112480E8882EAB
:100A9000912C18E0612E670CF701EA0DFB1DE95956
:100AA000FE4FE491172DC0E0D0E0CE2EDD24C4012E
:100AB0000C2E02C0959587950A94E2F78C219D2112
:100AC000892B21F0802F612F41E003C0802F612FFF
:100AD00040E00E94D50321961F5FC830D10539F749
:100AE000F701EA0DFB1DEF58FE4FE491162DC0E013
:100AF000D0E0CE2EDD24C4010C2E02C09595879542
:100B00000A94E2F78C219D21892B21F0802F612FFF
:100B100041E003C0802F612F40E00E94D503219661
:100B20001F5FC830D10539F70894E11CF11C0F5F35
:100B30008AE0E816F10409F0AFCFDF91CF911F9161
:100B40000F91FF90EF90DF90CF90BF90AF909F906C
:100B50008F907F906F9008957F928F929F92AF9227
:100B6000BF92CF92DF92EF92FF920F931F93CF939A
:100B7000DF93E82E762E842F81548A3118F080522C
:100B80008A3110F44F7119C0842F80538A3010F4C9
:100B9000415113C0403211F440E00FC04E3211F405
:100BA0004BE10BC0473211F44CE107C04A3311F45A
:100BB0004DE103C04E3309F44EE100E010E085E062
:100BC00048025001112490E4892E912CF801EA0D7D
:100BD000FB1DE859FF4FE491F72CC0E0D0E0CE2E8A
:100BE000DD24C4010C2E02C0959587950A94E2F786
:100BF0008C219D21892B21F08E2D6F2D41E003C08A
:100C00008E2D6F2D40E00E94D5032196F394C730BE
:100C1000D10539F70F5F1F4FE39405301105B1F689
:100C2000DF91CF911F910F91FF90EF90DF90CF90C8
:100C3000BF90AF909F908F907F900895CF92DF925A
:100C4000EF92FF920F931F93DF93CF93CDB7DEB751
:100C5000C854D0400FB6F894DEBF0FBECDBFE82E0B
:100C60000E945303DE011196E0E0F1E089E001907B
:100C70000D928150E1F7DE011A96EEE4F3E08FE386
:100C800001900D928150E1F710E06E010894C11CB3
:100C9000D11C0AC0C901880F991F820F931F880FAA
:100CA00060E00E94AC051F5F212F30E0F601E20FEB
:100CB000F31F4081442371F7FF242E2D30E0C9013A
:100CC000E3E0880F991FEA95E1F7820F931F8E01E9
:100CD0000F5F1F4F080F191F0AC0C901880F991F06
:100CE000820F931F880F68E00E94AC05F3942F2DAC
:100CF00030E0F801E20FF31F4185442371F733C060
:100D000086E0E81611F4EE2401C0E394FF248E2D52
:100D100090E08C0163E0000F111F6A95E1F7080F66
:100D2000191F0C0D1D1D0AC0C901880F991F820FC4
:100D3000931F880F68E00E94AC05F3942F2D30E0DC
:100D4000F801E20FF31F4185442371F766E970E073
:100D500080E090E00E94191E89EE93E00E94711DD0
:100D6000882329F0CDCF6E010894C11CD11C86EEDA
:100D700093E00E949B1D882379F38E2DC85BDF4F83
:100D80000FB6F894DEBF0FBECDBFCF91DF911F919C
:100D90000F91FF90EF90DF90CF900895AF92BF92A8
:100DA000CF92DF92EF92FF920F931F93DF93CF9337
:100DB000CDB7DEB7C956D0400FB6F894DEBF0FBE30
:100DC000CDBF182FE62EA42EB22E0E945303FE0193
:100DD000349686E6DF011D928A95E9F7A9E0B1E035
:100DE00089E00D9001928150E1F7FE013D9688E087
:100DF000DF011D928A95E9F7DE015596EAE1F1E0FF
:100E000089E001900D928150E1F7FE017E9688E025
:100E1000DF011D928A95E9F7DE019696EBE2F1E09B
:100E200089E001900D928150E1F7FE01BF9688E0C4
:100E3000DF011D928A95E9F7DE01D796ECE3F1E038
:100E400089E001900D928150E1F7FE01E05CFF4FD7
:100E500088E0DF011D928A95E9F7FE01E85BFF4F0C
:100E60009F014DE451E088E0DA010D90AD01D90118
:100E70000D929D018150C1F7389689E0DF011D92E6
:100E80008A95E9F7FE01E75AFF4F9F0140E051E0E4
:100E900089E0DA010D90AD01D9010D929D018150DB
:100EA000C1F7399688E0DF011D928A95E9F7FF24A2
:100EB000812F90E08C01B4E0000F111FBA95E1F78B
:100EC000080F191F6E010894C11CD11C0C0D1D1DAB
:100ED0000AC0C901880F991F820F931F880F60E015
:100EE0000E94AC05F3942F2D30E0F801E20FF31FC0
:100EF0004381442371F78E2D90E0B6014AE050E023
:100F00000E94C50280E068E049810E94AC0586E04D
:100F100068E04A810E94AC056CE271E080E090E0FC
:100F20000E94191E8E010F5F1F4F22C0EB1410F09C
:100F3000EA2C01C0E3948E2D90E0B8014AE050E025
:100F40000E94C50280E068E049810E94AC0586E00D
:100F500068E04A810E94AC0566E970E080E090E0BC
:100F60000E94191E89EE93E00E94711D8823F1F6FC
:100F700086EE93E00E949B1D8823A1F38E2DC75916
:100F8000DF4F0FB6F894DEBF0FBECDBFCF91DF911C
:100F90001F910F91FF90EF90DF90CF90BF90AF9097
:100FA0000895AF92BF92CF92DF92FF920F931F935B
:100FB000DF93CF93CDB7DEB7A2970FB6F894DEBF1D
:100FC0000FBECDBF809148039091490390930104D7
:100FD00080930004DE015396EDE8F3E080E1019098
:100FE0000D928150E1F780914A0390914B03892B38
:100FF00021F48EE591E098A38F8F81E090E09093AB
:10100000FF038093FE03FF24F39400E010E06E01E1
:101010000894C11CD11CEAE0AE2EB12CAC0EBD1E52
:1010200086EE93E00E949B1D882321F481E0F81650
:1010300009F06AC00E945303FF2049F480914803DD
:1010400090914903019690934903809348038091BE
:10105000480390914903089724F010924903109295
:101060004803C60166E671E00E94BE02E0914803B3
:10107000F0914903EE0FFF1FEC0DFD1D628973898E
:10108000C6010E94B302109148031F5F183008F098
:1010900010E0C50168E671E00E94BE02E12FF0E0B9
:1010A000EE0FFF1FEC0DFD1D62897389C5010E94C3
:1010B000B30210E00AC0C901880F991F820F931F65
:1010C000880F60E00E94AC051F5F212F30E0F60121
:1010D000E20FF31F4081442371F710E00AC0C901F9
:1010E000880F991F820F931F880F68E00E94AC053C
:1010F0001F5F212F30E0F501E20FF31F40814423F1
:1011000071F7FF2400E010E062E370E080E090E01F
:101110000E94191E0F5F1F4F083211050CF480CF7B
:1011200080914803909149030697A1F480914A0366
:1011300090914B0321E030E08227932790934B035B
:1011400080934A0380910004909101049093490395
:10115000809348038091480390914903079709F0D1
:101160004BC00E94530313E039C040914C0341022D
:10117000A001112481E064E028E00E94800428C0DE
:1011800080914C038F3029F410924C030E9453033A
:1011900003C08F5F80934C0340914C034102A00138
:1011A000112481E064E028E00E94800460914C03F7
:1011B000605680E00E94360360914C03605681E0E7
:1011C0000E94360366E970E080E090E00E94191EFC
:1011D00089EE93E00E94711D882391F686EE93E0DC
:1011E0000E949B1D882309F28091000490910104C4
:1011F0009093490380934803809148039091490359
:10120000049799F481E090E09093FB038093FA03B4
:101210008091F0039091F1039093FD038093FC0380
:10122000109249031092480304C01092FB031092DD
:10123000FA03A2960FB6F894DEBF0FBECDBFCF91D2
:10124000DF911F910F91FF90DF90CF90BF90AF90F3
:101250000895EF92FF921F93DF93CF93CDB7DEB740
:10126000A0970FB6F894DEBF0FBECDBFDE0111967A
:10127000EAE6F1E08CE001900D928150E1F71D86E5
:101280001E861F86188A10E07E010894E11CF11C5E
:1012900009C0880F991F880F991F8E5F61E00E9417
:1012A000A5041F5F812F90E0F701E80FF91F40812F
:1012B000442379F760EA7FE080E090E00E94191E05
:1012C0000E945303DE015196EAE7F1E087E00190C6
:1012D0000D928150E1F7FE01789689E0DF011D92C1
:1012E0008A95E9F710E0A1E1EA2EF12CEC0EFD1E43
:1012F00013C0C901F3E0880F991FFA95E1F7821B2B
:10130000930B8C5F65E00E94AC051F5F64EF71E09A
:1013100080E090E00E94191E212F30E0F701E20FDB
:10132000F31F4081442329F768EB7BE080E090E0E5
:101330000E94191E0E945303A0960FB6F894DEBFB8
:101340000FBECDBFCF91DF911F91FF90EF90089519
:101350009F92AF92BF92CF92DF92EF92FF920F9344
:101360001F93DF93CF93CDB7DEB7CA5BD0400FB6E4
:10137000F894DEBF0FBECDBF0E9453031091F2035D
:101380001150A090F4039090F6039A94FE01709689
:101390008FE3DF011D928A95E9F7AAE8B1E088E0C2
:1013A0000D9001928150E1F7188E87E595E6A4E64D
:1013B000B0E0898F9A8FAB8FBC8FFE017D9685E060
:1013C000DF011D928A95E9F7DE019296E3E9F1E0EB
:1013D00089E001900D928150E1F7DE019B96ECE9E6
:1013E000F1E087E001900D928150E1F71BAA1AAA63
:1013F000DE01D496E5EAF1E089E001900D9281509A
:10140000E1F7DE01DD96EEEAF1E087E001900D9272
:101410008150E1F7FE01EC5BFF4F118210829E01CB
:101420002A5B3F4FD901E7EBF1E087E001900D9295
:101430008150E1F7F90110861782DE01A15BBF4FF1
:101440008CE6FD0111928A95E9F79D0140EC51E08F
:1014500088E0FA010190AF01F90101929F018150EA
:10146000C1F718961C92DE01A85ABF4FE9ECF1E0D3
:1014700089E001900D928150E1F7FE01E15BFF4FA1
:101480009F012E5E3F4F42ED51E086E0DA010D9064
:10149000AD01D9010D929D018150C1F7789683E08D
:1014A000DF011D928A95E9F7FE01E15BFF4F9F0185
:1014B000255E3F4F4BED51E086E0DA010D90AD0126
:1014C000D9010D929D018150C1F7B19683E0DF01F2
:1014D0001D928A95E9F7FE01E15BFF4F8DE491E6ED
:1014E000A9E7B0E084A395A3A6A3B7A3B89685E027
:1014F000DF011D928A95E9F7B8979F01235D3F4F61
:1015000044EE51E085E0DA010D90AD01D9010D9274
:101510009D018150C1F712AA13AA14AA15AA9E010F
:10152000215B3F4FD901D696EDEEF1E085E00190C9
:101530000D928150E1F7F90113AE14AE15AE16AE5F
:10154000FE01E15BFF4F9F01215C3F4F46EF51E001
:1015500087E0DA010D90AD01D9010D929D01815016
:10156000C1F7EA5BFF4F118210829E0129563F4F5F
:10157000D901EFEFF1E085E001900D928150E1F7A4
:10158000F90115821682178210869E0120563F4F60
:10159000D901E8E0F2E088E001900D928150E1F796
:1015A000D90118961C92DE01A755BF4FE1E1F2E088
:1015B00089E001900D928150E1F7DE01AE54BF4FFA
:1015C000EAE1F2E089E001900D928150E1F760E0FC
:1015D00045E027E001E00E942A04F0E1EF2EF12C23
:1015E000EC0EFD1E89E0189FC0011124E80EF91EC3
:1015F000CC24DD2410E021C0812F60E045E027E00D
:1016000000E00E942A04812F60E04B2D0E94AC056F
:1016100086EE93E00E949B1D882309F018C189EE95
:1016200093E00E949B1D0894E11CF11C1A5F882323
:1016300009F00DC10894C11CD11CF701B080BB207A
:10164000D9F6C601880F991F8C0D9D1D880F991F13
:10165000803391053CF460E045E027E001E00E9422
:101660002A0406C06CE271E080E090E00E94191E3E
:1016700080E068E045E027E000E00E942A048A2D2F
:1016800090E0BE016F5F7F4F4AE050E00E94C502CC
:10169000DE011496E7ECF3E08CE001900D928150AE
:1016A000E1F7F1E0AF16A1F085E1A81689F0AFE10E
:1016B000AA1671F0B2E0AB1669F0E6E1AE1651F091
:1016C000F3E0AF1649F087E1A81631F013E005C04A
:1016D00010E003C011E001C012E080E068E0498141
:1016E0000E94AC05A9E0AA1518F066E0C62E0EC04F
:1016F00086E068E045E027E000E00E942A0486E0FA
:1017000068E04A810E94AC055CE0C52E8C2D68E043
:1017100045E027E000E00E942A04212F30E0C901C3
:10172000880F991F820F931F7E010894E11CF11C02
:10173000E80EF91EF701D3808C2D68E04D2D0E9434
:10174000AC051C2D1A5F812F68E045E027E00E9460
:101750002A04D7011496EC90812F68E04E2D0E9448
:10176000AC059CE0F92EFC0C8F2D68E045E027E0ED
:1017700001E00E942A040E94530380E060E0498156
:101780000E94AC0586E060E04A810E94AC058C2D89
:1017900060E04D2D0E94AC05812F60E04E2D0E942F
:1017A000AC058F2D60E045E027E000E00E942A04B0
:1017B0008FE4E82EF12CEC0EFD1E89E0989EC0010E
:1017C0001124E80EF91ECC24DD2410E01FC0812F67
:1017D00068E045E027E000E00E942A04812F68E0ED
:1017E0004B2D0E94AC0586EE93E00E949B1D882342
:1017F00071F589EE93E00E949B1D0894E11CF11C99
:101800001A5F882321F50894C11CD11CF701B08010
:10181000BB20E9F6C601880F991F8C0D9D1D880F0E
:10182000991F803391053CF468E045E027E002E031
:101830000E942A0406C068EE73E080E090E00E94F7
:10184000191E68EB7BE080E090E00E94191EC654F0
:10185000DF4F0FB6F894DEBF0FBECDBFCF91DF9143
:101860001F910F91FF90EF90DF90CF90BF90AF90BE
:101870009F9008950F931F93CF93DF93C0E0D0E024
:101880000C2FFE01E356FC4F1081812F61E00E9476
:10189000CF1E812F61E00E94F51E8BE061E00E9467
:1018A000CF1E8AE061E00E94CF1E8C2F61E00E9473
:1018B00036038C2F63E00E9436038C2F64E20E9473
:1018C000360310E0802F612F40E00E94B5031F5FB8
:1018D0001038C1F72196C230D10591F6DF91CF9132
:1018E0001F910F91089585E795E06CEE73E041E05C
:1018F0000E94451D08959F92AF92BF92CF92DF92B2
:10190000EF92FF920F931F930E9453030E94730C58
:101910006091EE031091F0030091F403D090F60370
:1019200080E040E02BE30E94CE06B82E81E0612FDC
:1019300040E027E10E94CE06C82E80E00E941E06ED
:10194000E82E84E0602F41E02FE10E94CE06982E21
:1019500083E06D2D41E02CE00E94CE06A82E82E0AF
:101960006DE04AE023E60E94CE06D82E05E715E09A
:10197000C8010E94FA1BC80160E070E040E050E03E
:101980000E94021CC80161E070E04B2D50E00E94F3
:10199000021CC80162E070E04C2D50E00E94021C65
:1019A000FF240894E11CF11CC80163E070E0A7016A
:1019B0000E94021CC80164E070E0492D50E00E94C2
:1019C000021CC80165E070E04A2D50E00E94021C34
:1019D000C80166E070E04D2D50E00E94021CC80175
:1019E0000E94F51B0E945303809100049091010412
:1019F00090934903809348031F910F91FF90EF90BC
:101A0000DF90CF90BF90AF909F9008952F923F921C
:101A10004F925F927F928F929F92AF92BF92CF929E
:101A2000DF92EF92FF920F931F93DF93CF93CDB787
:101A3000DEB7C95FD0400FB6F894DEBF0FBECDBF92
:101A40000E945303FE01FC968EEBDF011D928A95E6
:101A5000E9F78FE69EE6A5E6B0E08CAF9DAFAEAFAE
:101A6000BFAF26E0FE01E05CFF4FDF01822F1D9239
:101A70008A95E9F7FE01EA5BFF4F84E797E7AFE657
:101A8000B0E081939193A193B193DF011D922A95C8
:101A9000E9F79E01205B3F4FD901E1E3F2E086E0E8
:101AA00001900D928150E1F7F9011682178210869C
:101AB0001186FE01E65AFF4F9F014BE352E085E09D
:101AC000DA010D90AD01D9010D929D018150C1F750
:101AD000359685E0DF011D928A95E9F7FE01EC5904
:101AE000FF4F9F0145E452E085E0DA010D90AD0122
:101AF000D9010D929D018150C1F7359685E0DF0136
:101B00001D928A95E9F7FE01E259FF4F83E799E6B6
:101B1000A8E7B0E081939193A193B19386E0DF01B0
:101B20001D928A95E9F79E0128583F4FD901EFE4AD
:101B3000F2E086E001900D928150E1F7F901168202
:101B40001782108611869E012E573F4FD901E9E575
:101B5000F2E086E001900D928150E1F7D9011696EE
:101B60001D921D921D921C921997FE01E457FF4F82
:101B70009F0143E652E085E0DA010D90AD01D90105
:101B80000D929D018150C1F7359685E0DF011D92D0
:101B90008A95E9F7FE01EA56FF4F84E795E6AEE63F
:101BA000B0E081939193A193B19386E0DF011D9200
:101BB0008A95E9F7FE01E056FF4F9F014DE652E09E
:101BC00087E0DA010D90AD01D9010D929D018150A0
:101BD000C1F7379683E0DF011D928A95E9F7FE0190
:101BE000E655FF4F9F0147E752E087E0DA010D908D
:101BF000AD01D9010D929D018150C1F7379683E067
:101C0000DF011D928A95E9F79E012C543F4FD901BF
:101C1000E1E8F2E089E001900D928150E1F7F901ED
:101C200011869E0122543F4FD901EBE8F2E089E092
:101C300001900D928150E1F7D90119961C929E01F5
:101C400028533F4FD901E5E9F2E088E001900D9279
:101C50008150E1F7F901118610869E012E523F4F07
:101C6000D901EFE9F2E088E001900D928150E1F7AF
:101C7000D90119961C921E921897DE01A452BF4FEB
:101C8000E9EAF2E08AE001900D928150E1F79E01CD
:101C90002A513F4FD901E3EBF2E089E001900D9228
:101CA0008150E1F7F90111869E0120513F4FD90182
:101CB000EDEBF2E089E001900D928150E1F7D9015E
:101CC00019961C92FE01799683E2DF011D928A9596
:101CD000E9F784E795E6AEE6B0E0898F9A8FAB8F9F
:101CE000BC8FFE017D9683E0DF011D928A95E9F7A6
:101CF000DE019096E7ECF2E087E001900D928150D2
:101D0000E1F7DE019796EEECF2E087E001900D92AC
:101D10008150E1F7DE019E96E5EDF2E086E001906C
:101D20000D928150E1F71CAADE01D596ECEDF2E0B0
:101D300086E001900D928150E1F71BAE7090EE03AA
:101D4000442455245E010894A11CB11C1DE0C12E41
:101D5000D12CCC0EDD1EBCE38B2E912C8C0E9D1E47
:101D6000A9E12A2E312C2C0E3D1E0E94730C86EE0A
:101D700093E00E949B1D882319F00E94D1076EC139
:101D800089EE93E00E949B1D882339F00E94A809E8
:101D90000E948C030E94060D61C18091EC0380FDBE
:101DA00003C08DE061E002C08DE060E00E94F51E9E
:101DB0004114510451F0272D30E08091EE039091B1
:101DC000EF032817390709F438C17090EE0310911A
:101DD000F0031D3008F01C50112309F41CE0872D7E
:101DE0006AE00E94CB22E92EFF24B9E0B71540F14A
:101DF000C7010197BC01F3E0660F771FFA95E1F781
:101E0000880F991F680F791F680D791DC5010E9401
:101E1000BE02C50163E272E00E94B302812F90E02E
:101E20000197BC0153E0660F771F5A95E1F7880FC1
:101E3000991F680F791F680D791DC6010E94BE02A7
:101E4000EAE07E1669F4C501BE016A567F4F0E9422
:101E5000BE02C50163E272E00E94B302812F25C079
:101E6000872D6AE00E94CB220E94CB22092F992362
:101E700009F473C0812F90E0E114F10409F44BC020
:101E80000197BC0133E0660F771F3A95E1F7880FA1
:101E9000991F680F791F680D791DC5010E94BE0248
:101EA000872D8B50893080F4872D90E00197BC01FD
:101EB00003E0660F771F0A95E1F7880F991F680FF7
:101EC000791F680D791D44C0802F90E00197BC01F7
:101ED000B3E0660F771FBA95E1F7681B790B620DC7
:101EE000731DC6010E94BE02C60168E671E00E9431
:101EF000B302C7010197BC01A3E0660F771FAA9543
:101F0000E1F7880F991F680F791F680D791DC601C9
:101F10000E94B30220C00197BC01E3E0660F771F67
:101F2000EA95E1F7880F991F680F791F680D791DF1
:101F3000C5010E94BE02802F90E00197BC0143E0E2
:101F4000660F771F4A95E1F7681B790B620D731DC9
:101F5000C6010E94BE0290E019C0EF28E1F7812F70
:101F600090E00197BC0133E0660F771F3A95E1F7E7
:101F7000880F991F680F791F680D791DC5010E9490
:101F8000BE02C60169E272E0E4CF9F5F292F30E014
:101F9000F501E20FF31F80818823B9F781E090E01B
:101FA000821B930B880F991F880F991F8F9662E0F1
:101FB00070E00E94D722F62E90E001C09F5F292F8B
:101FC00030E0F601E20FF31F80818823B9F781E04A
:101FD00090E0821B930B880F991F880F991F8F9693
:101FE00062E070E00E94D722062F0E948C0310E06E
:101FF00009C0880F991F880F991F8F0D62E00E94FA
:10200000A5041F5F812F90E0F501E80FF91F4081C3
:10201000442379F710E009C0880F991F880F991F92
:10202000800F69E00E94A5041F5F812F90E0F601F8
:10203000E80FF91F4081442379F762E370E080E004
:1020400090E00E94191E0894411C511CF8E84F169C
:10205000F3E15F0609F089CE0E948C03C750DF4F81
:102060000FB6F894DEBF0FBECDBFCF91DF911F91A9
:102070000F91FF90EF90DF90CF90BF90AF909F9027
:102080008F907F905F904F903F902F9008952F9268
:102090003F924F925F926F927F928F929F92AF92F8
:1020A000BF92CF92DF92EF92FF920F931F93DF9335
:1020B000CF93CDB7DEB76D970FB6F894DEBF0FBEE6
:1020C000CDBF0E94530380E060E04FE220E100E0DA
:1020D0000E942A040E9453030E94730C10E088E1BE
:1020E000612F41E00E94D5031F5F1031C1F72AE044
:1020F0002D8B2C8B45E050E05F874E875D874C87AA
:102100005D834C835B874A8711E01F821E8280912A
:10211000EC0380FD03C08DE061E002C08DE060E073
:102120000E94F51E86EE93E00E949B1D882319F005
:102130000E94D107C6C489EE93E00E949B1D8823AC
:1021400039F00E94A8090E948C030E944710B9C46C
:10215000112309F4C2C08D896C8940E00E94D50327
:102160000091EE031091F0031D3078F080914A0346
:1021700090914B03BC01A4EFBFEF6A9FC0016B9F1E
:10218000900D7A9F900D1124180F112361F4209166
:102190004A0330914B03C901880F991F820F931F87
:1021A000182F110F110F812F90E0BE016F5F7F4F2D
:1021B0004AE050E00E94C5021A3020F489818A83E7
:1021C000B0E3B9838EE060E049810E94A50482E11A
:1021D00060E04A810E94A504802F90E0BE016F5FFD
:1021E0007F4F4AE050E00E94C5020A3020F4898106
:1021F0008A8320E329838CE160E049810E94A50461
:1022000080E260E04A810E94A50464E070E080E022
:1022100090E02CE030E040E050E00E9436217B016D
:102220008C0160E070E080E090E022E030E040E08F
:1022300050E00E94362116161706180619064CF0B3
:1022400040E050E060E87FEB488B598B6A8B7B8BDA
:1022500008C060E070E080E89FE3688B798B8A8B30
:102260009B8B60E070E080E090E022E030E040E0B6
:1022700050E00E94362116161706180619065CF063
:102280000F2EF0E02F2EF0E03F2EF0E04F2EFFEB70
:102290005F2EF02D0AC00F2EF0E02F2EF0E03F2E23
:1022A000F0E04F2EFFE35F2EF02DC801B7010E9432
:1022B000F8216E8B7F8B888F998F6CED75E080E0B5
:1022C00090E00E94191E80E090E0A8EBB1E48A8FB4
:1022D0009B8FAC8FBD8F198618860E94730C8091DE
:1022E000EC039091ED03CB9769F48091EE0390910C
:1022F000EF038B3391050CF0DEC391E0998702C0A8
:10230000A1E0A8876EE170E080E090E029E230E093
:1023100040E050E00E9436210E94F8219B01AC0170
:102320006A8D7B8D8C8D9D8D0E94C121882341F407
:102330006E897F89888D998D0E94C5217D836C83EC
:1023400068E070E080E090E023E130E040E050E0C1
:102350000E9436210E94F8219B01AC016A8D7B8D81
:102360008C8D9D8D0E94C121882341F46E897F89C7
:10237000888D998D0E94C5217B876A876A8D7B8DA8
:102380008C8D9D8D20E030E048EB51E40E94C1210E
:10239000882309F097C0688979898A899B8920E018
:1023A00030E040E050E00E94C12188230CF08AC058
:1023B00042013101EE88FF88088D198DAA8CBB8CF3
:1023C000CC8CDD8C28C0C801B701A40193010E9408
:1023D0005D217B018C0120E030E040E050E00E9474
:1023E000C121181654F4C801B70120E030E040E7DD
:1023F00051E40E94A822882324F097FA909497F839
:102400009094C601B501288939894A895B890E945F
:102410005D215B016C01C601B50120E030E040E0C8
:1024200050E40E94A822181654F4C601B50120E019
:1024300030E044E352E40E94C12187FDC4CFC801CB
:10244000B7010E94CA21162FB985B130F9F469305D
:1024500068F060E070E080E090E023E030E040E091
:1024600050E00E9436217D836C8329C360E070E0D8
:1024700080E090E023E030E040E050E00E94362130
:102480009B01285F3F4F3D832C8319C360E070E0C0
:1024900080E090E026E030E040E050E00E9436210D
:1024A000812F90E0861B970B97FD0AC09D838C833C
:1024B0000B970CF4ADC04AE050E05D834C83A8C09C
:1024C0001D821C826A8D7B8D8C8D9D8D20E030E07D
:1024D00048EC51E40E94C121882309F099C0688921
:1024E00079898A899B8920E030E040E050E00E94B1
:1024F000A82218160CF08CC042013101EE88FF882A
:10250000088D198DAA8CBB8CCC8CDD8C28C0C801A1
:10251000B701A40193010E945D217B018C0120E0A1
:1025200030E040E050E00E94C121181654F4C80188
:10253000B70120E030E040E751E40E94A822882360
:1025400024F097FA909497F89094C601B5012889E1
:1025500039894A895B890E945D215B016C01C60152
:10256000B50120E030E040E050E40E94A8221816B7
:1025700054F4C601B50120E030E044E352E40E9487
:10258000C12187FDC4CFC801B7010E94CA21162FFF
:1025900058855130F9F4693068F060E070E080E00F
:1025A00090E023E030E040E050E00E9436217B875D
:1025B0006A870EC060E070E080E090E023E030E0E9
:1025C00040E050E00E943621DB011896BB87AA87C5
:1025D00018861EC060E070E080E090E026E030E009
:1025E00040E050E00E943621212F30E0261B370BBF
:1025F0003B872A8737FF03C01B861A8609C04A8596
:102600005B854B30510524F06AE070E07B876A8778
:102610008E859F85AC81BD81A817B90734F4181643
:1026200019068CF401979F878E872E853F854C81F4
:102630005D81241735073CF42A30310524F42F5FDF
:102640003F4F3F872E87EE84FF84F094E194F1089A
:10265000F39410E056E0E516F10448F481E0612FB0
:1026600041E00E94D50380E0612F41E008C081E095
:10267000612F40E00E94D50380E0612F40E00E947E
:10268000D5031F5F0894E11CF11C103119F76C850C
:102690007D858A859B85861797073CF41616170655
:1026A0008CF4615070407D876C87AC85BD852A8530
:1026B0003B85A217B30734F4AA30B1051CF4119678
:1026C000BD87AC87EC84FD84F094E194F108F39429
:1026D00010E036E0E316F10448F48EE2612F41E0A9
:1026E0000E94D5038FE2612F41E008C08EE2612F86
:1026F00040E00E94D5038FE2612F40E00E94D503A5
:102700001F5F0894E11CF11C103119F76A8D7B8D55
:102710008C8D9D8D288939894A895B890E945D212C
:102720006A8F7B8F8C8F9D8F6E897F89888D998D25
:10273000A20191010E945D216E8B7F8B888F998F02
:1027400020E030E040E050E00E94C12118166CF01B
:1027500057FA509457F8509440E050E060E070E031
:102760004E8B5F8B688F798F18C06E897F89888DBB
:10277000998D20E030E040E751E40E94A8228823B0
:1027800064F057FA509457F8509460E070E080E796
:1027900091E46E8B7F8B888F998F6A8D7B8D8C8D6A
:1027A0009D8D0E94C5217B0172E0E716F10409F0BE
:1027B0005BC06E897F89888D998D0E94C5218E8529
:1027C0009F85681779070CF4EFC005968617970761
:1027D0000CF4EAC060E070E080E090E023E030E0DC
:1027E00040E050E00E943621611571058105910598
:1027F00009F45FC060E070E080E090E022E030E04B
:1028000040E050E00E9436214E855F854230510500
:102810004CF048305105BCF4662321F0613009F0DA
:10282000C3C011C061E070E080E090E023E030E0E0
:1028300040E050E00E943621AC81BD81A60FB71F59
:10284000BD83AC8368C061E070E080E090E023E08D
:1028500030E040E050E00E9436214C815D81461B13
:10286000570B5D834C8383C07DE2E716F10409F0CA
:102870009BC06E897F89888D998D0E94C5218C852A
:102880009D85681779070CF48FC005968617970702
:102890000CF48AC060E070E080E090E023E030E07B
:1028A00040E050E00E9436216115710581059105D7
:1028B00051F4288939894A895B895058288B398B8A
:1028C0004A8B5B8B71C060E070E080E090E022E0BA
:1028D00030E040E050E00E9436214C855D8542307A
:1028E00051054CF04830510594F5662321F06130D4
:1028F00009F05AC02CC061E070E080E090E023E075
:1029000030E040E050E00E943621AA85BB85A60F4A
:10291000B71FBB87AA87288939894A895B8950589C
:10292000288B398B4A8B5B8BC201B10120E030E0F0
:1029300040E050E40E94C1218823B4F5C201B101F6
:102940002DEC3CEC4CE45EE30E945D212BC061E089
:1029500070E080E090E023E030E040E050E00E9452
:1029600036214A855B85461B570B5B874A876889FA
:1029700079898A899B899058688B798B8A8B9B8B04
:10298000C201B1012DEC3CEC4CE45EE30E94A822B4
:10299000181654F4C201B1012DEC3CEC4CE45EE39A
:1029A0000E945C211B012C016A8D7B8D8C8D9D8D7D
:1029B00020E030E040E05FE30E945D210E94C521FD
:1029C000162F6E897F89888D998D20E030E040E058
:1029D0005FE30E945D210E94C521062FE2E0F4E042
:1029E0008081982F9F708295807F982B919374E0BF
:1029F000E23CF707A9F7412F4851483118F0412F21
:102A000050E001C051E0802F90E0440F440F9C0142
:102A10003595279535952795420F252F30E0A0E66F
:102A2000B0E02A9FF0012B9FF00D3A9FF00D11248A
:102A3000E40FF11DEE5FFB4F208130E0837090705A
:102A400048E050E002C0559547958A95E2F7CA01E3
:102A500090E028233923232B31F08D896C8940E0C5
:102A60000E94D5030CC0812F602F41E00E94D50346
:102A70008D896C8940E00E94D5031D8B0C8BE1147D
:102A8000F10429F010E05FE2E516F10409F411E029
:102A900064E170E080E090E00E94191E6E817F8109
:102AA0006F5F7F4F7F836E836858734109F02FCB30
:102AB0000E948C0306C0CB9709F422CC23CC198644
:102AC000A7CD6D960FB6F894DEBF0FBECDBFCF91E8
:102AD000DF911F910F91FF90EF90DF90CF90BF900B
:102AE000AF909F908F907F906F905F904F903F90AE
:102AF0002F9008959F92AF92BF92CF92DF92EF9264
:102B0000FF920F931F93DF93CF9300D00F92CDB717
:102B1000DEB70E9453030091EE03EE24FF246E0102
:102B20000894C11CD11CA0E39A2EF4EFAF2EFFEF46
:102B3000BF2E0E94730C8091EC0380FD03C08DE0DA
:102B400061E002C08DE060E00E94F51E86EE93E039
:102B50000E949B1D882319F00E94D107A0C089EE16
:102B600093E00E949B1D882339F00E94A8090E94CF
:102B70008C030E947A1593C0E114F10451F0202FC8
:102B800030E08091EE039091EF032817390709F4A4
:102B900075C00091EE031091F0031D3068F0809134
:102BA0004A0390914B039C012A9DC0012B9D900DDF
:102BB0003A9D900D1124180F112361F420914A03BE
:102BC00030914B03C901880F991F820F931F182F53
:102BD000110F110F812F90E0B6014AE050E00E94E2
:102BE000C5021A3018F489818A83998280E061E0F5
:102BF00049810E9419058CE061E04A810E94190513
:102C000087E164E041E00E94D50387E165E041E0AF
:102C10000E94D50388E164E041E00E94D50388E189
:102C200065E041E00E94D50387E16AE041E00E944F
:102C3000D50387E16BE041E00E94D50388E16AE0BB
:102C400041E00E94D50388E16BE041E00E94D5039A
:102C5000802F90E0B6014AE050E00E94C5020A30A1
:102C600018F489818A8399828AE161E049810E940E
:102C7000190586E261E04A810E94190562E370E06D
:102C800080E090E00E94191E0894E11CF11C38E8D5
:102C9000E31633E1F30609F04CCF0E948C030F904A
:102CA0000F900F90CF91DF911F910F91FF90EF90B8
:102CB000DF90CF90BF90AF909F9008952F923F925A
:102CC0004F925F926F927F928F929F92AF92BF923C
:102CD000CF92DF92EF92FF920F931F93DF93CF93E8
:102CE000CDB7DEB7C458D0400FB6F894DEBF0FBEE4
:102CF000CDBFDE01A05CBF4FEBEAF3E08CE10190B9
:102D00000D928150E1F7DE01A45ABF4FE3EEF2E0ED
:102D100085E201900D928150E1F76090EE030E94F0
:102D20005303CF57DF4F19821882C158D04080E338
:102D3000282E312C2C0E3D1EA101405F5F4FCD5738
:102D4000DF4F59834883C358D0400E94730C809151
:102D5000EC0380FD03C08DE061E002C08DE060E027
:102D60000E94F51E86EE93E00E949B1D882309F0C9
:102D70008EC189EE93E00E949B1D882339F00E944A
:102D8000A8090E948C030E947A15A9C1CF57DF4F72
:102D900088819981C158D040892B11F421010AC042
:102DA000262D30E08091EE039091EF03281739072C
:102DB000A9F77CC1842D8219D2018D932D01CD57A5
:102DC000DF4FE881F981C358D040AE17BF0791F7B4
:102DD000710100E010E00E94420260E170E0601BBF
:102DE000710B0E94D722FC01E00FF11FD7019C91CB
:102DF000E20DF31D80818D937D0190830F5F1F4F46
:102E00000F30110541F76090EE03F090F003BCE045
:102E1000BF1578F480914A0390914B0324EF3FEF64
:102E2000FC01E29FC001E39F900DF29F900D1124E1
:102E3000F80EFF2061F420914A0330914B03C90141
:102E4000880F991F820F931FF82EFF0CFF0CD09054
:102E5000F203E090F4038E01005E1F4F60E070E02B
:102E600080E090E024E130E040E050E00E94362134
:102E70006D5FD8016D938D01A215B30579F78F2D84
:102E800090E0BE016F5F7F4F4AE050E00E94C502B4
:102E9000B9E0BF1520F089818A8380E38983F980B6
:102EA000CA80862D90E0BE016F5F7F4F4AE050E000
:102EB0000E94C502E9E0E61520F089818A8380E35B
:102EC000898309811A818E2D90E0BE016F5F7F4F4B
:102ED0004AE050E00E94C502F9E0FE1520F0898129
:102EE0008A8380E38983DE011496EFE9F3E08CE0C6
:102EF00001900D928150E1F721E0E216A1F045E149
:102F0000E41689F05FE1E51671F082E0E81669F0F9
:102F100096E1E91651F0A3E0EA1649F0B7E1EB16A5
:102F200031F023E005C020E003C021E001C022E031
:102F3000F88AC98A8AE38A8B0B8B1C8B90E29D8B63
:102F40009E8B9F8BDA94ED2DF0E0EE0FFF1FEE0FBE
:102F5000FF1FA1E0B0E0AC0FBD1FAE0FBF1FDF969B
:102F60008C91DF97888FA05CBF4F8C91898F41E057
:102F700050E04C0F5D1FE40FF51FEF5BFF4F8081AA
:102F80008A8F9B8F89818C8F8A818D8F822F90E091
:102F9000FC01EE0FFF1FE80FF91FE40FF51F8381FF
:102FA0008E8F84818F8F77247FC0D6012C9128301B
:102FB00028F0F8E09F2EE8E08E2E02C099248824A5
:102FC000022F10E070E2A72EB12CAC0EBD1EA00E99
:102FD000B11EF501F080F1E0FF1510F560E070E042
:102FE00080E090E024E230E040E050E00E943621B2
:102FF000AB01BC01980129193109C901880F991F3A
:10300000820F931FECE5F0E0EC0FFD1FE40FF51FBE
:10301000880F682D40810E94AC05FA94D501FC927E
:1030200080E2E82EF12CEC0EFD1EE00EF11EF70101
:1030300080818130B1F4980129193109C901880FC3
:10304000991F820F931FE0E1F0E0EC0FFD1FE00FEE
:10305000F11F880F682D40810E94AC05D7011C929A
:103060007394E0E2F0E0EC0FFD1F0E0F1F1FD8017C
:103070008C91882331F464E070E080E090E00E945D
:10308000191E86EE93E00E949B1D882319F00E9472
:10309000D10725C00894C11CD11CC414D50409F063
:1030A00084CFBFE0B71510F061017FCF62E370E01D
:1030B00080E090E00E94191ECF57DF4FE881F98130
:1030C000C158D0403196CF57DF4FF983E883C158BC
:1030D000D040E858F34109F038CE0E948C03CC5719
:1030E000DF4F0FB6F894DEBF0FBECDBFCF91DF919B
:1030F0001F910F91FF90EF90DF90CF90BF90AF9016
:103100009F908F907F906F905F904F903F902F9007
:103110000895CF93DF938091FA039091FB03892B5D
:10312000E1F10E94730CC091FC03D091FD038091EA
:10313000F0039091F103C817D90779F562E070E0C8
:1031400080E090E024E030E040E050E00E94362152
:10315000CE01860F971F9093FD038093FC03489741
:1031600074F061E070E080E090E022E030E040E068
:1031700050E00E9436217093FD036093FC0360E0F1
:1031800070E080E090E024E030E040E050E00E9419
:1031900036217093490360934803809148039091CE
:1031A000490382309105A1F0833091052CF40097FA
:1031B00049F00197A9F409C08330910561F00597A2
:1031C00079F40CC00E947A150BC00E94471008C009
:1031D0000E94060D05C00E945E1602C00E947B0C74
:1031E0008091FE039091FF03892B39F40E948C0398
:1031F0000E94A8090E948C0304C01092FF03109241
:10320000FE03DF91CF91089581E161E00E94CF1E1E
:1032100081E161E00E94F51E80E161E00E94CF1E25
:1032200080E160E00E94F51E89E096E040E855E20A
:1032300060E070E00E94D11F0E943A0C81E00E9481
:10324000AD1E0E94542160914C03605680E00E94A4
:10325000360360914C03605681E00E9436030E9461
:1032600029090E94730C8091F0039091F1039093CF
:10327000FD038093FC03089581E08093070560932C
:10328000E404109205051092060508959091E20459
:103290008091E304981710F080E00895E92FF0E0A2
:1032A000EE53FB4F80819F5F9093E2040895089551
:1032B000DF93CF930F92CDB7DEB769838091070577
:1032C000882389F080910605803290F4809105056D
:1032D000E82FF0E0EB51FB4F60838F5F8093050593
:1032E0008093060505C0CE01019661E00E94371A61
:1032F0000F90CF91DF9108950E9458190895809101
:10330000E40465EE74E04091060521E00E94F419A2
:103310001092050510920605109207050895413296
:1033200008F040E2862F62EC74E00E94BD19109212
:10333000E2048093E30408950E948F190895109287
:10334000E2041092E30410920505109206050E9413
:10335000AA19089510920905449A459AE9EBF0E0FC
:1033600080818E7F808380818D7F808388E48093BD
:10337000B80085E48093BC000895982F413210F086
:1033800040E030C0809109058823E1F781E0809317
:1033900009058FEF8093740510922F0541504093DB
:1033A00030054F5F990F916090930A0585EE8093E9
:1033B000BC00809109058130E1F380912F058417CD
:1033C00010F440912F0520E030E00AC0FB01E20F2D
:1033D000F31FD901A15FBA4F8C9180832F5F3F4FBC
:1033E0002417A0F3842F08951F93582F122F4132D2
:1033F00010F081E03AC0809109058823E1F782E06E
:10340000809309058FEF8093740510922F054093E8
:103410003005AFE0B5E0FB0102C081918D938E2FA6
:10342000861B8417D0F3852F90E0880F991F809317
:103430000A0585EE8093BC00112321F080910905D7
:103440008230E1F3809174058F3F11F480E00DC06C
:1034500080917405803211F482E007C08091740578
:10346000803311F084E001C083E01F910895482F5C
:10347000613210F081E0089580910905843011F0E7
:1034800082E0089560935205A1E3B5E0842F9C018A
:10349000F90102C081918D938E2F841B8617D0F382
:1034A00080E008951F920F920FB60F9211242F9370
:1034B0003F934F935F936F937F938F939F93AF93BC
:1034C000BF93EF93FF938091B90090E0887F907055
:1034D0008036910509F4DCC081369105CCF588323F
:1034E000910509F47BC089329105B4F480319105CE
:1034F00009F46FC0813191053CF4009709F431C1A2
:10350000089709F039C165C08831910509F466C092
:10351000809709F031C17DC08034910509F49FC0C6
:103520008134910544F48033910509F47DC0C89736
:1035300009F022C184C08035910509F484C0883522
:10354000910509F491C08834910509F015C198C01E
:103550008839910509F4FDC089399105ECF4883763
:10356000910509F495C0893791054CF48836910589
:1035700009F48EC08037910509F0FEC089C08838F3
:10358000910509F4E6C08039910509F487C08038B7
:10359000910509F0F1C082C0803B910509F4B0C0EB
:1035A000813B91054CF4803A910509F489C0883A31
:1035B000910509F0E1C0A4C0803C910509F4CDC09B
:1035C000883C910509F4C9C0883B910509F0D4C035
:1035D000ACC080910A058093BB00B9C090912F05C3
:1035E00080913005981768F490912F05E92FF0E04D
:1035F000E15FFA4F80818093BB009F5F90932F051E
:10360000A6C085ED8093BC008091BC0084FDFCCFFA
:10361000B1C080E28093740585ED8093BC008091F9
:10362000BC0084FDFCCFA6C080E38093740585EDCB
:103630008093BC008091BC0084FDFCCF9BC088E3DC
:10364000809374058AC080912F059091BB00E82F6C
:10365000F0E0E15FFA4F90838F5F80932F059091A8
:103660002F058091300571C080912F059091BB008E
:10367000E82FF0E0E15FFA4F90838F5F80932F0592
:1036800085ED8093BC008091BC0084FDFCCF72C0AE
:1036900083E0809309051092730559C080917305EA
:1036A000803208F056C0809173059091BB00E82FDE
:1036B000F0E0ED5AFA4F90838F5F8093730547C017
:1036C00080917305803230F4E0917305F0E0ED5A9B
:1036D000FA4F108285ED8093BC008091BC0084FD80
:1036E000FCCF1092090560917305E0910D05F091F2
:1036F0000E0583E595E070E00995109273052DC0E5
:1037000084E0809309051092510510925205E091D2
:103710000B05F0910C05099580915205882329F439
:1037200081E0809352051092310590915105E92F67
:10373000F0E0EF5CFA4F80818093BB009F5F909335
:1037400051059091510580915205981710F485EC20
:1037500001C085E88093BC000FC085EC8093BC005D
:1037600009C01092740585ED8093BC008091BC0067
:1037700084FDFCCF10920905FF91EF91BF91AF91AD
:103780009F918F917F916F915F914F913F912F9179
:103790000F900FBE0F901F9018950F931F93CF930C
:1037A000DF938C0188E095E068E670E00E943C19A8
:1037B00088E095E060E070E00E947C19C0E0D0E015
:1037C000F801EC0FFD1F88E095E060810E94581918
:1037D0002196C730D105A1F788E095E00E947F19B6
:1037E000DF91CF911F910F910895FC0110820E94EB
:1037F000CD1B0895FC01808180688083CF010E94E9
:10380000CD1B0895CF93DF93EC01FA01633071056E
:1038100009F458C0643071054CF46130710551F100
:1038200062307105DCF5672B71F089C06530710578
:1038300009F460C0653071050CF449C0663071054B
:1038400009F07DC06AC04C33510508F078C0CA0148
:103850006AE070E00E94D722262F2295207FCF01B8
:103860006AE070E00E94D722280F88818078822B3E
:10387000888365C04C33510508F061C0CA016AE015
:1038800070E00E94D722262F2295207FCF016AE088
:1038900070E00E94D722280F298351C0483151057A
:1038A00008F04DC0CA016AE070E00E94D722262FBE
:1038B0002295207FCF016AE070E00E94D722280F76
:1038C0002A833DC048305105D0F54B8338C0403283
:1038D0005105A8F5CA016AE070E00E94D722262FA0
:1038E0002295207FCF016AE070E00E94D722280F46
:1038F0002C8325C04D30510510F5CA016AE070E0F7
:103900000E94D722262F2295207FCF016AE070E007
:103910000E94D722280F2D8312C04336510578F418
:10392000CA016AE070E00E94D722262F2295207FEC
:10393000CF016AE070E00E94D722280F2E83CE01CB
:103940000E94CD1BDF91CF9108950F931F93CF93CA
:10395000DF938C0188E095E068E670E00E943C19F6
:1039600088E095E060E070E00E947C1988E095E0D6
:103970000E947F1988E095E068E670E047E050E03B
:103980000E949C19C0E0D0E088E095E00E944619B2
:10399000F801EC0FFD1F80832196C730D105A1F7F8
:1039A000DF91CF911F910F9108950F931F93CF93A4
:1039B000DF938C01EB01442311F00E94A51CC3305E
:1039C000D10521F1C430D1054CF4C130D105A1F0AD
:1039D000C230D105C4F4CD2B61F008C0C530D1058B
:1039E000F9F0C530D105CCF0269791F14FEF5FEF9C
:1039F00046C0F801208102C0F801218130E0C901F0
:103A00008077907013C0F80122810CC0F801838187
:103A1000482F50E04770507032C0F801248102C036
:103A2000F801258130E0C90180739070A4E095957C
:103A30008795AA95E1F7AC01F3E0440F551FFA957D
:103A4000E1F7880F991F480F591F2F70307015C06C
:103A5000F8018681482F50E04F7050704053584F06
:103A600082958F7090E09C0173E0220F331F7A954E
:103A7000E1F7880F991F280F391F420F531FCA0102
:103A8000DF91CF911F910F910895EF92FF920F93C5
:103A90001F93CF93DF937C01162F072F442311F040
:103AA0000E94A51C812F902F9C018901C0E0D0E0CD
:103AB000C701BE0140E00E94D51CF801819391939B
:103AC0008F012196C730D10599F7DF91CF911F91D2
:103AD0000F91FF90EF90089588E095E00E949F1964
:103AE0000895CF93DF93EC018A8180FF02C082604A
:103AF00001C08D7F8A8388810E944D1F298130E01B
:103B00004A818217930711F44E7F01C041604A83B6
:103B10004A81242F30E0C901959587958227932704
:103B200080FF02C0446001C04B7F4A838A8181705C
:103B3000DF91CF910895CF93DF93EC010E94711D27
:103B4000882339F08A8190E0969587959695879598
:103B50008170DF91CF910895FC0181E081838081A4
:103B600061E00E94F51E08951F93CF93DF93EC014F
:103B7000862F142F688360E00E94CF1E112311F45A
:103B8000198203C0CE010E94AC1D1A82898188234C
:103B900019F481E08A8301C01A82DF91CF911F91CD
:103BA00008951F920F920FB60F9211242F933F93F7
:103BB0008F939F93AF93BF938091800590918105E0
:103BC000A0918205B0918305309184050196A11DD5
:103BD000B11D232F2D5F2D3720F02D570196A11DEC
:103BE000B11D209384058093800590938105A09357
:103BF0008205B093830580917C0590917D05A0910D
:103C00007E05B0917F050196A11DB11D80937C05B5
:103C100090937D05A0937E05B0937F05BF91AF91F2
:103C20009F918F913F912F910F900FBE0F901F90FA
:103C300018959B01AC017FB7F89480917C05909119
:103C40007D05A0917E05B0917F0566B5A89B05C056
:103C50006F3F19F00196A11DB11D7FBFBA2FA92F8B
:103C6000982F8827860F911DA11DB11D62E0880F36
:103C7000991FAA1FBB1F6A95D1F7BC012DC0FFB7C2
:103C8000F89480917C0590917D05A0917E05B0917E
:103C90007F05E6B5A89B05C0EF3F19F00196A11D71
:103CA000B11DFFBFBA2FA92F982F88278E0F911D06
:103CB000A11DB11DE2E0880F991FAA1FBB1FEA9545
:103CC000D1F7861B970B885E9340C8F22150304095
:103CD0004040504068517C4F211531054105510548
:103CE00071F60895789484B5826084BD84B581604E
:103CF00084BD85B5826085BD85B5816085BDEEE6F4
:103D0000F0E0808181608083E1E8F0E010828081D2
:103D100082608083808181608083E0E8F0E0808140
:103D200081608083E1EBF0E0808184608083E0EB60
:103D3000F0E0808181608083EAE7F0E08081846048
:103D400080838081826080838081816080838081A4
:103D5000806880831092C1000895982F8E3008F0FB
:103D60009E50977080914D038295880F880F807CBC
:103D7000892B80937C0080917A00806480937A0004
:103D800080917A0086FDFCCF2091780040917900E7
:103D9000942F80E030E0282B392BC9010895482F5B
:103DA00050E0CA01835A9C4FFC012491475B5C4F51
:103DB000FA0184918823C1F0E82FF0E0EE0FFF1F95
:103DC000E55DFC4FA591B491662341F49FB7F8944B
:103DD0008C91209582238C939FBF08959FB7F89470
:103DE0008C91822B8C939FBF0895482F50E0CA017D
:103DF0008F589C4FFC012491CA01835A9C4FFC01AF
:103E00003491475B5C4FFA019491992309F444C0C3
:103E1000222351F1233071F0243028F42130A1F015
:103E2000223011F514C02630B1F02730C1F0243013
:103E3000D9F404C0809180008F7703C08091800006
:103E40008F7D8093800010C084B58F7702C084B5C9
:103E50008F7D84BD09C08091B0008F7703C08091B1
:103E6000B0008F7D8093B000E92FF0E0EE0FFF1FD0
:103E7000EB5CFC4FA591B491662341F49FB7F89495
:103E80008C91309583238C939FBF08959FB7F894AE
:103E90008C91832B8C939FBF0895682F70E0CB018A
:103EA0008F589C4FFC012491CB01835A9C4FFC01FD
:103EB0004491675B7C4FFB019491992319F420E0B6
:103EC00030E03CC0222351F1233071F0243028F43B
:103ED0002130A1F0223011F514C02630B1F0273086
:103EE000C1F02430D9F404C0809180008F7703C0E2
:103EF000809180008F7D8093800010C084B58F7783
:103F000002C084B58F7D84BD09C08091B0008F77D9
:103F100003C08091B0008F7D8093B000892F90E026
:103F2000880F991F815C9C4FFC01A591B4918C91E5
:103F300020E030E0842311F021E030E0C901089551
:103F40001F920F920FB60F9211242F933F934F930E
:103F50008F939F93EF93FF934091C600E0910506E6
:103F6000F091060631969F012F773070319780913E
:103F70000706909108062817390739F0EB57FA4FD2
:103F800040833093060620930506FF91EF919F91A1
:103F90008F914F913F912F910F900FBE0F901F90D7
:103FA0001895CF93DF93EC019A01AB01E885F98571
:103FB000203081EE380780E0480780E0580709F498
:103FC00049C081E090E00A8802C0880F991F0A94D6
:103FD000E2F7808360E079E08DE390E00E940C23BB
:103FE0002150304040405040CA01B90122E030E049
:103FF00040E050E00E940C23EC81FD813083EE8193
:10400000FF812083EA85FB85208141E050E0CA01E1
:104010000E8402C0880F991F0A94E2F7282B208390
:10402000EA85FB852081CA010F8402C0880F991F91
:104030000A94E2F7282B2083EA85FB858081088893
:1040400002C0440F551F0A94E2F7842B8083DF914E
:10405000CF910895108220E130E0CECFDC0112969E
:10406000ED91FC911397E058FF4F219131918081A0
:104070009181281B390B2F773070C9010895DC011D
:104080001296ED91FC911397EE57FF4F20813181ED
:1040900092918291E058F0408217930719F42FEF24
:1040A0003FEF05C0E20FF31F8081282F30E0C901E8
:1040B0000895DC011296ED91FC911397DF01AE5744
:1040C000BF4F2D913C911197E058FF4F8081918116
:1040D000E058F0408217930719F42FEF3FEF0BC021
:1040E000E20FF31F80812F5F3F4F2F7730702D93AA
:1040F0003C93282F30E0C9010895DC011296ED9120
:10410000FC911397EE57FF4F808191819293829398
:104110000895FC01A085B18521898C9190E0022E43
:1041200002C0959587950A94E2F780FFF6CF048444
:10413000F585E02D6083089587ED93E090930A065E
:104140008093090685E895E090930C0680930B0612
:1041500085EC90E090930E0680930D0684EC90E041
:104160009093100680930F0680EC90E090931206D7
:104170008093110681EC90E09093140680931306CF
:1041800086EC90E0909316068093150684E0809369
:10419000170683E08093180687E08093190685E070
:1041A00080931A0681E080931B0608950E94721E78
:1041B0000E9404190E948918FDCF0F931F93CF937B
:1041C000DF938C01EB0109C02196D801ED91FC91A0
:1041D0000190F081E02DC801099568816623A1F75F
:1041E000DF91CF911F910F910895EF92FF920F935E
:1041F0001F93CF93DF938C017B01EA010CC0D701A1
:104200006D917D01D801ED91FC910190F081E02D3F
:10421000C80109952197209791F7DF91CF911F91C0
:104220000F91FF90EF900895EF92FF920F931F93DD
:104230007B018C01611571058105910529F420E050
:1042400030E040E050E00BC00E94A502A8019701B9
:104250000E940C23AC01CB01DA019C01AD01B90134
:10426000CA011F910F91FF90EF900895EF92FF9276
:104270000F931F937B018C016217730784079507C7
:1042800064F4261B370B480B590BCA01B9010E9475
:104290001421E60EF71E081F191FB701C8011F9150
:1042A0000F91FF90EF900895009729F0BC0180E0F6
:1042B00090E00E94AA0208955058BB27AA270ED06A
:1042C0000DC1FED030F003D120F031F49F3F11F446
:1042D0001EF4F3C00EF4E095E7FBE9C0E92F0FD11F
:1042E00080F3BA17620773078407950718F071F413
:1042F0009EF527C10EF4E0950B2EBA2FA02D0B01D1
:10430000B90190010C01CA01A0011124FF27591B1A
:1043100099F0593F50F4503E68F11A16F040A22F20
:10432000232F342F4427585FF3CF46953795279591
:10433000A795F0405395C9F77EF41F16BA0B620B90
:10434000730B840BBAF09150A1F0FF0FBB1F661FD7
:10435000771F881FC2F70EC0BA0F621F731F841F1A
:1043600048F4879577956795B795F7959E3F08F040
:10437000B3CF9395880F08F09927EE0F97958795FF
:10438000089571D008F481E0089504D06894B111C3
:10439000D9C00895BCD088F09F5790F0B92F9927C5
:1043A000B751A0F0D1F0660F771F881F991F1AF040
:1043B000BA95C9F712C0B13081F0C3D0B1E0089509
:1043C000C0C0672F782F8827B85F39F0B93FCCF38A
:1043D000869577956795B395D9F73EF49095809536
:1043E000709561957F4F8F4F9F4F0895E89409C056
:1043F00097FB3EF490958095709561957F4F8F4F18
:104400009F4F9923A9F0F92F96E9BB279395F6952D
:10441000879577956795B795F111F8CFFAF4BB0FAB
:1044200011F460FF1BC06F5F7F4F8F4F9F4F16C00F
:10443000882311F096E911C0772321F09EE8872F99
:10444000762F05C0662371F096E8862F70E060E055
:104450002AF09A95660F771F881FDAF7880F9695CE
:10446000879597F90895990F0008550FAA0BE0E872
:10447000FEEF16161706E807F907C0F01216130626
:10448000E407F50798F0621B730B840B950B39F466
:104490000A2661F0232B242B252B21F408950A26CC
:1044A00009F4A140A6958FEF811D811D089597F90C
:1044B0009F6780E870E060E008959FEF80EC0895CA
:1044C00000240A94161617061806090608950024F3
:1044D0000A9412161306140605060895092E03946D
:1044E000000C11F4882352F0BB0F40F4BF2B11F4E1
:1044F00060FF04C06F5F7F4F8F4F9F4F089557FD40
:104500009058440F551F59F05F3F71F04795880F41
:1045100097FB991F61F09F3F79F0879508951216D8
:1045200013061406551FF2CF4695F1DF08C0161684
:1045300017061806991FF1CF869571056105089435
:104540000895E894BB2766277727CB0197F908954C
:104550008ADF08F48FEF0895629FD001739FF00106
:10456000829FE00DF11D649FE00DF11D929FF00D03
:10457000839FF00D749FF00D659FF00D9927729F3A
:10458000B00DE11DF91F639FB00DE11DF91FBD01C5
:10459000CF0111240895991B79E004C0991F961743
:1045A00008F0961B881F7A95C9F78095089597FBA8
:1045B000092E07260AD077FD04D049D006D0002066
:1045C0001AF4709561957F4F0895F6F7909581954F
:1045D0009F4F0895A1E21A2EAA1BBB1BFD010DC01F
:1045E000AA1FBB1FEE1FFF1FA217B307E407F507A3
:1045F00020F0A21BB30BE40BF50B661F771F881F7F
:10460000991F1A9469F760957095809590959B0114
:10461000AC01BD01CF01089597FB092E05260ED0F0
:1046200057FD04D0D7DF0AD0001C38F450954095D0
:10463000309521953F4F4F4F5F4F0895F6F7909576
:104640008095709561957F4F8F4F9F4F0895AA1B5E
:10465000BB1B51E107C0AA1FBB1FA617B70710F06D
:10466000A61BB70B881F991F5A95A9F7809590959F
:10467000BC01CD010895EE0FFF1F0590F491E02DD0
:1046800009942F923F924F925F926F927F928F92F6
:104690009F92AF92BF92CF92DF92EF92FF920F93D1
:1046A0001F93CF93DF93CDB7DEB7CA1BDB0B0FB6DB
:1046B000F894DEBF0FBECDBF09942A883988488898
:1046C0005F846E847D848C849B84AA84B984C8842E
:1046D000DF80EE80FD800C811B81AA81B981CE0F25
:1046E000D11D0FB6F894DEBF0FBECDBFED0108950A
:0446F000F894FFCF6C
:1046F400444159204E414D4500534554204D494EA7
:104704005300000000000000000053455420484FAF
:104714005552000000000000000000534554205989
:1047240045415200000000000000000053455420A1
:104734004D4E544800000000000000000053455452
:104744002044415900000000000000000000313204
:1047540020486F7572003E002000444144275320D6
:10476400434C4F434B00000000004641544845521F
:1047740000000000000000000000547565736461CF
:1047840079000054687572736461790046726964D3
:104794006179000000536174757264617900537526
:1047A4006E6461790000004D6F6E646179000000F1
:1047B4004A616E7561727900004665627275617254
:1047C40079004D6172636800000000417072696C89
:1047D400000000004A756E6500000000004A756C18
:1047E4007900000000004175677573740000005380
:1047F40065707400000000004F63746F626572009E
:10480400004E6F76656D62657200446563656D6226
:104814006572002050415354004F27434C4F434B83
:104824000074687265650000000000666F757200B0
:104834000000000000666976650000000000007357
:104844006576656E000000000065696768740000A5
:104854000000006E696E65000000000000656C6574
:1048640076656E000000007477656C766500000064
:1048740000746869727465656E0000666F757274A1
:1048840065656E00006669667465656E0000007398
:1048940069787465656E000000736576656E74658D
:1048A400656E00656967687465656E00006E696EA3
:1048B400657465656E00007477656E74790074685C
:1048C4006972747900666F7274790000666966743F
:1048D4007900004142434445464748494A4B4C4DC0
:1048E4004E4F505152535455565758595A313233EA
:1048F40034353637383930004E756D626572730061
:10490400506F6E6700576F726473004A756D626C06
:10491400650052616E646F6D0053657420436C6B67
:1049240000323420486F75720042726967687400FF
:1049340001000000010000000100010007015455BE
:10494400455344415920005745442020202020004D
:104954005448555253444159004652494441592000
:10496400200053415455524441590053554E44413B
:10497400592020004D4F4E44415920200008031077
:104984000315031B032203290331033903040573AD
:1049940074006E64007264007468005455450057D6
:1049A400454400544855004652490053415400536D
:1049B400554E004D4F4E007374006E6400726400D7
:1049C400746800000000008920DD20F5202E2059A5
:0649D400203F207D2000C1
:00000001FF
